 cspddk

 Timestamp is 4fb05c78 (Mon May 14 13:14:32 2012)

 Preferred load address is 10000000

 Start         Length     Name                   Class
 0001:00000000 00000004H .CRT$XCA                CODE
 0001:00000004 00000004H .CRT$XCZ                CODE
 0001:00000008 00000004H .CRT$XIA                CODE
 0001:0000000c 00000004H .CRT$XIZ                CODE
 0001:00000010 00000004H .CRT$XPA                CODE
 0001:00000014 00000004H .CRT$XPZ                CODE
 0001:00000018 00000004H .CRT$XTA                CODE
 0001:0000001c 00000004H .CRT$XTZ                CODE
 0001:00000020 00001bdaH .rdata                  CODE
 0001:00001bfc 00000023H .rdata$debug            CODE
 0001:00001c20 00008c64H .text                   CODE
 0001:0000a884 00000018H .xdata                  CODE
 0001:0000a89c 00000014H .idata$2                CODE
 0001:0000a8b0 00000014H .idata$3                CODE
 0001:0000a8c4 000000d4H .idata$4                CODE
 0001:0000a998 0000000cH .idata$6                CODE
 0001:0000a9b0 000004ebH .edata                  CODE
 0002:00000000 000000d4H .idata$5                DATA
 0002:000000d8 00000044H .data                   DATA
 0002:00000120 00000098H .bss                    DATA
 0003:00000000 00000418H .pdata                  DATA

  Address         Publics by Value              Rva+Base       Lib:Object

 0000:00000000       ___safe_se_handler_table   00000000     <absolute>
 0000:00000000       ___safe_se_handler_count   00000000     <absolute>
 0001:00000000       __xc_a                     10001000     corelib0:crt0init.obj
 0001:00000004       __xc_z                     10001004     corelib0:crt0init.obj
 0001:00000008       __xi_a                     10001008     corelib0:crt0init.obj
 0001:0000000c       __xi_z                     1000100c     corelib0:crt0init.obj
 0001:00000010       __xp_a                     10001010     corelib0:crt0init.obj
 0001:00000014       __xp_z                     10001014     corelib0:crt0init.obj
 0001:00000018       __xt_a                     10001018     corelib0:crt0init.obj
 0001:0000001c       __xt_z                     1000101c     corelib0:crt0init.obj
 0001:00000040       ??_C@_1EI@FEPNPNPF@?$AAC?$AAl?$AAo?$AAc?$AAk?$AAA?$AAl?$AAl?$AAo?$AAc?$AA?3?$AA?5?$AA?5?$AAM?$AAm?$AAM?$AAa?$AAp?$AAI?$AAo?$AAS?$AAp?$AAa?$AAc?$AAe?$AA?5?$AAf?$AAa?$AAi?$AAl?$AAe?$AAd@ 10001040     ddk_mx25_topaz_v1:soc_ddk_clk.obj
 0001:00000088       ??_C@_1CI@OHCJFJPM@?$AAE?$AAR?$AAR?$AAO?$AAR?$AA?3?$AA?5?$AA?$CF?$AAs?$AA?5?$AAl?$AAi?$AAn?$AAe?$AA?5?$AA?$CF?$AAd?$AA?3?$AA?5?$AA?$AA@ 10001088     ddk_mx25_topaz_v1:soc_ddk_clk.obj
 0001:000000b0       ??_C@_1FK@FNONLNGN@?$AA?$CF?$AAs?$AA?3?$AA?5?$AAD?$AAE?$AAB?$AAU?$AAG?$AAC?$AAH?$AAK?$AA?5?$AAf?$AAa?$AAi?$AAl?$AAe?$AAd?$AA?5?$AAi?$AAn?$AA?5?$AAf?$AAi?$AAl?$AAe?$AA?5?$AA?$CF?$AAs?$AA?5?$AAa@ 100010b0     ddk_mx25_topaz_v1:soc_ddk_clk.obj
 0001:0000010c       ??_C@_1O@JEGGABPH@?$AAC?$AAS?$AAP?$AAD?$AAD?$AAK?$AA?$AA@ 1000110c     ddk_mx25_topaz_v1:soc_ddk_clk.obj
 0001:00000120       ??_C@_1ME@OCDNAJAG@?$AAC?$AA?3?$AA?2?$AAW?$AAI?$AAN?$AAC?$AAE?$AAR?$AAO?$AAO?$AAT?$AAS?$AA?2?$AAT?$AAo?$AAp?$AAa?$AAz?$AA?2?$AAW?$AAI?$AAN?$AAC?$AAE?$AA6?$AA0?$AA0?$AA?2?$AAP?$AAL?$AAA@ 10001120     ddk_mx25_topaz_v1:soc_ddk_clk.obj
 0001:000001e8       ??_C@_1ME@JPMIENNJ@?$AAC?$AA?3?$AA?2?$AAW?$AAI?$AAN?$AAC?$AAE?$AAR?$AAO?$AAO?$AAT?$AAS?$AA?2?$AAT?$AAo?$AAp?$AAa?$AAz?$AA?2?$AAW?$AAI?$AAN?$AAC?$AAE?$AA6?$AA0?$AA0?$AA?2?$AAP?$AAL?$AAA@ 100011e8     ddk_mx25_topaz_v1:ddk_gpio.obj
 0001:000002b0       ??_C@_1EG@HEFOPIHA@?$AAG?$AAp?$AAi?$AAo?$AAA?$AAl?$AAl?$AAo?$AAc?$AA?3?$AA?5?$AA?5?$AAM?$AAm?$AAM?$AAa?$AAp?$AAI?$AAo?$AAS?$AAp?$AAa?$AAc?$AAe?$AA?5?$AAf?$AAa?$AAi?$AAl?$AAe?$AAd?$AA?$CB@ 100012b0     ddk_mx25_topaz_v1:ddk_gpio.obj
 0001:000002f8       ??_C@_1EO@FDEPDNPK@?$AAI?$AAo?$AAm?$AAu?$AAx?$AAA?$AAl?$AAl?$AAo?$AAc?$AA?3?$AA?5?$AA?5?$AAV?$AAi?$AAr?$AAt?$AAu?$AAa?$AAl?$AA?5?$AAm?$AAa?$AAp?$AAp?$AAi?$AAn?$AAg?$AA?5?$AAf?$AAa?$AAi@ 100012f8     ddk_mx25_topaz_v1:soc_ddk_iomux.obj
 0001:00000348       ??_C@_1MM@FPBDMGFP@?$AAC?$AA?3?$AA?2?$AAW?$AAI?$AAN?$AAC?$AAE?$AAR?$AAO?$AAO?$AAT?$AAS?$AA?2?$AAT?$AAo?$AAp?$AAa?$AAz?$AA?2?$AAW?$AAI?$AAN?$AAC?$AAE?$AA6?$AA0?$AA0?$AA?2?$AAP?$AAL?$AAA@ 10001348     ddk_mx25_topaz_v1:soc_ddk_iomux.obj
 0001:00000414       ??_C@_1DE@GMFODGCD@?$AAS?$AAd?$AAm?$AAa?$AAS?$AAe?$AAt?$AAC?$AAh?$AAa?$AAn?$AAD?$AAe?$AAs?$AAc?$AA?5?$AAf?$AAa?$AAi?$AAl?$AAe?$AAd?$AA?$CB?$AA?$AN?$AA?6?$AA?$AA@ 10001414     ddk_mx25_topaz_v1:ddk_sdmav2.obj
 0001:00000448       ??_C@_1DA@HDPMDGLM@?$AAN?$AAo?$AA?5?$AAa?$AAv?$AAa?$AAi?$AAl?$AAa?$AAb?$AAl?$AAe?$AA?5?$AAc?$AAh?$AAa?$AAn?$AAn?$AAe?$AAl?$AA?$CB?$AA?$AN?$AA?6?$AA?$AA@ 10001448     ddk_mx25_topaz_v1:ddk_sdmav2.obj
 0001:00000478       ??_C@_1MM@NICEDNOK@?$AAC?$AA?3?$AA?2?$AAW?$AAI?$AAN?$AAC?$AAE?$AAR?$AAO?$AAO?$AAT?$AAS?$AA?2?$AAT?$AAo?$AAp?$AAa?$AAz?$AA?2?$AAW?$AAI?$AAN?$AAC?$AAE?$AA6?$AA0?$AA0?$AA?2?$AAP?$AAL?$AAA@ 10001478     ddk_mx25_topaz_v1:ddk_sdmav2.obj
 0001:00000544       ??_C@_1DK@FOEAIIIE@?$AAC?$AAh?$AAa?$AAn?$AAn?$AAe?$AAl?$AA?5?$AAv?$AAa?$AAl?$AAi?$AAd?$AAa?$AAt?$AAi?$AAo?$AAn?$AA?5?$AAf?$AAa?$AAi?$AAl?$AAe?$AAd?$AA?$CB?$AA?$AN?$AA?6?$AA?$AA@ 10001544     ddk_mx25_topaz_v1:ddk_sdmav2.obj
 0001:00000580       ??_C@_1DI@IIDNCCFN@?$AAB?$AAS?$AAP?$AAS?$AAd?$AAm?$AAa?$AAA?$AAl?$AAl?$AAo?$AAc?$AAC?$AAh?$AAa?$AAi?$AAn?$AA?5?$AAf?$AAa?$AAi?$AAl?$AAe?$AAd?$AA?$CB?$AA?$AN?$AA?6?$AA?$AA@ 10001580     ddk_mx25_topaz_v1:ddk_sdmav2.obj
 0001:000005b8       ??_C@_1CO@MINJNIPA@?$AAC?$AAa?$AAn?$AAn?$AAo?$AAt?$AA?5?$AAk?$AAi?$AAl?$AAl?$AA?5?$AAc?$AAh?$AAa?$AAn?$AAn?$AAe?$AAl?$AA?$CB?$AA?$AN?$AA?6?$AA?$AA@ 100015b8     ddk_mx25_topaz_v1:ddk_sdmav2.obj
 0001:000005e8       ??_C@_1CG@BCAFLFJD@?$AAI?$AAn?$AAv?$AAa?$AAl?$AAi?$AAd?$AA?5?$AAc?$AAh?$AAa?$AAn?$AAn?$AAe?$AAl?$AA?$CB?$AA?$AN?$AA?6?$AA?$AA@ 100015e8     ddk_mx25_topaz_v1:ddk_sdmav2.obj
 0001:00000610       ??_C@_1CI@NLJOHANF@?$AAI?$AAn?$AAv?$AAa?$AAl?$AAi?$AAd?$AA?5?$AAB?$AAD?$AA?5?$AAi?$AAn?$AAd?$AAe?$AAx?$AA?$CB?$AA?$AN?$AA?6?$AA?$AA@ 10001610     ddk_mx25_topaz_v1:ddk_sdmav2.obj
 0001:00000638       ??_C@_1DO@GBCIMEAG@?$AAC?$AAa?$AAn?$AAn?$AAo?$AAt?$AA?5?$AAl?$AAo?$AAa?$AAd?$AA?5?$AAc?$AAh?$AAa?$AAn?$AAn?$AAe?$AAl?$AA?5?$AAc?$AAo?$AAn?$AAt?$AAe?$AAx?$AAt?$AA?$CB?$AA?$AN?$AA?6?$AA?$AA@ 10001638     ddk_mx25_topaz_v1:ddk_sdmav2.obj
 0001:00000678       ??_C@_1EK@EDMAEBMC@?$AAC?$AAa?$AAn?$AAn?$AAo?$AAt?$AA?5?$AAi?$AAn?$AAi?$AAt?$AAi?$AAa?$AAl?$AAi?$AAz?$AAe?$AA?5?$AAc?$AAh?$AAa?$AAn?$AAn?$AAe?$AAl?$AA?5?$AAc?$AAo?$AAn?$AAt?$AAe?$AAx@ 10001678     ddk_mx25_topaz_v1:ddk_sdmav2.obj
 0001:000006c8       ??_C@_1EK@IEHBFKHA@?$AAC?$AAh?$AAa?$AAi?$AAn?$AA?5?$AAs?$AAt?$AAa?$AAt?$AAu?$AAs?$AA?5?$AAc?$AAo?$AAu?$AAl?$AAd?$AA?5?$AAn?$AAo?$AAt?$AA?5?$AAb?$AAe?$AA?5?$AAc?$AAl?$AAe?$AAa?$AAr?$AAe@ 100016c8     ddk_mx25_topaz_v1:ddk_sdmav2.obj
 0001:00000714       ??_C@_1CM@DDOONFFB@?$AAC?$AAh?$AAa?$AAn?$AAn?$AAe?$AAl?$AA?5?$AAn?$AAo?$AAt?$AA?5?$AAo?$AAp?$AAe?$AAn?$AAe?$AAd?$AA?$CB?$AA?$AN?$AA?6?$AA?$AA@ 10001714     ddk_mx25_topaz_v1:ddk_sdmav2.obj
 0001:00000740       ??_C@_1EC@HDIDMHOC@?$AAS?$AAd?$AAm?$AAa?$AAS?$AAt?$AAo?$AAp?$AAC?$AAh?$AAa?$AAn?$AA?3?$AA?5?$AA?5?$AAI?$AAn?$AAv?$AAa?$AAl?$AAi?$AAd?$AA?5?$AAc?$AAh?$AAa?$AAn?$AAn?$AAe?$AAl?$AA?$AN?$AA?6@ 10001740     ddk_mx25_topaz_v1:ddk_sdmav2.obj
 0001:00000788       ??_C@_1IO@IAEKHNEP@?$AAW?$AAA?$AAR?$AAN?$AAI?$AAN?$AAG?$AA?3?$AA?5?$AA?5?$AAS?$AAD?$AAM?$AAA?$AA?5?$AAh?$AAo?$AAs?$AAt?$AA?5?$AAs?$AAh?$AAa?$AAr?$AAe?$AAd?$AA?5?$AAr?$AAe?$AAg?$AAi?$AAo@ 10001788     ddk_mx25_topaz_v1:ddk_sdmav2.obj
 0001:00000818       ??_C@_1BE@KFLCBOIG@?$AAM?$AAU?$AAT?$AAE?$AAX?$AA_?$AAA?$AAC?$AAR?$AA?$AA@ 10001818     ddk_mx25_topaz_v1:ddk_sdmav2.obj
 0001:0000082c       ??_C@_1CM@FONMNFCK@?$AAC?$AAr?$AAe?$AAa?$AAt?$AAe?$AAM?$AAu?$AAt?$AAe?$AAx?$AA?5?$AAf?$AAa?$AAi?$AAl?$AAe?$AAd?$AA?$CB?$AA?$AN?$AA?6?$AA?$AA@ 1000182c     ddk_mx25_topaz_v1:ddk_sdmav2.obj
 0001:00000858       ??_C@_1BG@GPGAHAMG@?$AAM?$AAU?$AAT?$AAE?$AAX?$AA_?$AAS?$AAD?$AAM?$AAA?$AA?$AA@ 10001858     ddk_mx25_topaz_v1:ddk_sdmav2.obj
 0001:00000870       ??_C@_1DO@NANMFPJP@?$AAS?$AAD?$AAM?$AAA?$AA?5?$AAM?$AAC?$AA0?$AAP?$AAT?$AAR?$AA?5?$AAn?$AAo?$AAt?$AA?5?$AAi?$AAn?$AAi?$AAt?$AAi?$AAa?$AAl?$AAi?$AAz?$AAe?$AAd?$AA?$CB?$AA?$AN?$AA?6?$AA?$AA@ 10001870     ddk_mx25_topaz_v1:ddk_sdmav2.obj
 0001:000008b0       ??_C@_1CO@FMOECGMA@?$AAM?$AAm?$AAM?$AAa?$AAp?$AAI?$AAo?$AAS?$AAp?$AAa?$AAc?$AAe?$AA?5?$AAf?$AAa?$AAi?$AAl?$AAe?$AAd?$AA?$CB?$AA?$AN?$AA?6?$AA?$AA@ 100018b0     ddk_mx25_topaz_v1:ddk_sdmav2.obj
 0001:000008e0       ??_C@_1FG@NHFMOGCL@?$AAC?$AAh?$AAa?$AAn?$AA?5?$AA0?$AA?5?$AAb?$AAu?$AAf?$AAf?$AAe?$AAr?$AA?5?$AAd?$AAe?$AAs?$AAc?$AAr?$AAi?$AAp?$AAt?$AAo?$AAr?$AA?5?$AAi?$AAn?$AAc?$AAu?$AAr?$AAr?$AAe@ 100018e0     ddk_mx25_topaz_v1:ddk_sdmav2.obj
 0001:00000938       ??_C@_1FE@JFANIPC@?$AAC?$AAh?$AAa?$AAn?$AA?5?$AA0?$AA?5?$AAb?$AAu?$AAf?$AAf?$AAe?$AAr?$AA?5?$AAd?$AAe?$AAs?$AAc?$AAr?$AAi?$AAp?$AAt?$AAo?$AAr?$AA?5?$AAn?$AAo?$AAt?$AA?5?$AAp?$AAr?$AAo@ 10001938     ddk_mx25_topaz_v1:ddk_sdmav2.obj
 0001:0000098c       ??_C@_1DI@NPAFFBOK@?$AAC?$AAh?$AAa?$AAn?$AA?5?$AA0?$AA?5?$AAc?$AAa?$AAn?$AAn?$AAo?$AAt?$AA?5?$AAb?$AAe?$AA?5?$AAs?$AAt?$AAa?$AAr?$AAt?$AAe?$AAd?$AA?$CB?$AA?$AN?$AA?6?$AA?$AA@ 1000198c     ddk_mx25_topaz_v1:ddk_sdmav2.obj
 0001:000009c4       ??_C@_1DG@CMHJFFKC@?$AAN?$AAo?$AA?5?$AAu?$AAn?$AAu?$AAs?$AAe?$AAd?$AA?5?$AAc?$AAh?$AAa?$AAn?$AAn?$AAe?$AAl?$AA?5?$AAf?$AAo?$AAu?$AAn?$AAd?$AA?$CB?$AA?$AN?$AA?6?$AA?$AA@ 100019c4     ddk_mx25_topaz_v1:ddk_sdmav2.obj
 0001:000009fc       ??_C@_1CG@EDBHHEHJ@?$AAC?$AAl?$AAo?$AAc?$AAk?$AAA?$AAl?$AAl?$AAo?$AAc?$AA?5?$AAf?$AAa?$AAi?$AAl?$AAe?$AAd?$AA?$CB?$AA?$AA@ 100019fc     ddk_mx25_topaz_v1:cspddk.obj
 0001:00000a24       ??_C@_1CG@HJKJMKDE@?$AAI?$AAo?$AAm?$AAu?$AAx?$AAA?$AAl?$AAl?$AAo?$AAc?$AA?5?$AAf?$AAa?$AAi?$AAl?$AAe?$AAd?$AA?$CB?$AA?$AA@ 10001a24     ddk_mx25_topaz_v1:cspddk.obj
 0001:00000a4c       ??_C@_1CE@EFFDAGJH@?$AAG?$AAp?$AAi?$AAo?$AAA?$AAl?$AAl?$AAo?$AAc?$AA?5?$AAf?$AAa?$AAi?$AAl?$AAe?$AAd?$AA?$CB?$AA?$AA@ 10001a4c     ddk_mx25_topaz_v1:cspddk.obj
 0001:00000a70       ??_C@_1CE@OLEDCPDM@?$AAS?$AAd?$AAm?$AAa?$AAA?$AAl?$AAl?$AAo?$AAc?$AA?5?$AAf?$AAa?$AAi?$AAl?$AAe?$AAd?$AA?$CB?$AA?$AA@ 10001a70     ddk_mx25_topaz_v1:cspddk.obj
 0001:00000a98       ??_C@_1LC@MICAPKBE@?$AAC?$AA?3?$AA?2?$AAW?$AAI?$AAN?$AAC?$AAE?$AAR?$AAO?$AAO?$AAT?$AAS?$AA?2?$AAT?$AAo?$AAp?$AAa?$AAz?$AA?2?$AAW?$AAI?$AAN?$AAC?$AAE?$AA6?$AA0?$AA0?$AA?2?$AAP?$AAL?$AAA@ 10001a98     ddk_mx25_topaz_v1:cspddk.obj
 0001:00000b4c       ??_C@_1CC@OCAHOLEK@?$AAS?$AAd?$AAm?$AAa?$AAI?$AAn?$AAi?$AAt?$AA?5?$AAf?$AAa?$AAi?$AAl?$AAe?$AAd?$AA?$CB?$AA?$AA@ 10001b4c     ddk_mx25_topaz_v1:cspddk.obj
 0001:00000d80       g_pSdmaBaseRegPA           10001d80     ddk_mx25_topaz_v1:soc_ddk_sdma.obj
 0001:00000e18       ??_C@_1BO@ICEODACO@?$AAE?$AAV?$AAE?$AAN?$AAT?$AA_?$AAS?$AAE?$AAT?$AAP?$AAO?$AAI?$AAN?$AAT?$AA?$AA@ 10001e18     ddk_clk:ddk_clk.obj
 0001:00000e38       ??_C@_1CM@PPPGIKAO@?$AAC?$AAr?$AAe?$AAa?$AAt?$AAe?$AAE?$AAv?$AAe?$AAn?$AAt?$AA?5?$AAf?$AAa?$AAi?$AAl?$AAe?$AAd?$AA?$CB?$AA?$AN?$AA?6?$AA?$AA@ 10001e38     ddk_clk:ddk_clk.obj
 0001:00000e64       ??_C@_1CE@KCPPCGKP@?$AAE?$AAV?$AAE?$AAN?$AAT?$AA_?$AAD?$AAV?$AAF?$AAC?$AA_?$AAW?$AAO?$AAR?$AAK?$AAE?$AAR?$AA?$AA@ 10001e64     ddk_clk:ddk_clk.obj
 0001:00000e88       ??_C@_1FE@PIPHAHND@?$AAB?$AAS?$AAP?$AAC?$AAl?$AAo?$AAc?$AAk?$AAA?$AAl?$AAl?$AAo?$AAc?$AA?3?$AA?5?$AAs?$AAh?$AAo?$AAu?$AAl?$AAd?$AA?5?$AAm?$AAa?$AAp?$AA?5?$AAg?$AA_?$AAp?$AAC?$AAR?$AAM@ 10001e88     ddk_clk:ddk_clk.obj
 0001:00000ee0       ??_C@_1EO@BABGMAOC@?$AAB?$AAS?$AAP?$AAC?$AAl?$AAo?$AAc?$AAk?$AAA?$AAl?$AAl?$AAo?$AAc?$AA?3?$AA?5?$AA?5?$AAM?$AAm?$AAM?$AAa?$AAp?$AAI?$AAo?$AAS?$AAp?$AAa?$AAc?$AAe?$AA?5?$AAf?$AAa?$AAi@ 10001ee0     ddk_clk:ddk_clk.obj
 0001:00000f30       ??_C@_1KG@EMPAJGPO@?$AAC?$AA?3?$AA?2?$AAW?$AAI?$AAN?$AAC?$AAE?$AAR?$AAO?$AAO?$AAT?$AAS?$AA?2?$AAT?$AAo?$AAp?$AAa?$AAz?$AA?2?$AAW?$AAI?$AAN?$AAC?$AAE?$AA6?$AA0?$AA0?$AA?2?$AAP?$AAL?$AAA@ 10001f30     ddk_clk:ddk_clk.obj
 0001:00000fd8       dmaDriverPath              10001fd8     ddk_dma:ddk_dma.obj
 0001:00000ff0       dmaDriverName              10001ff0     ddk_dma:ddk_dma.obj
 0001:00001008       ??_C@_1II@DMGIDHM@?$AAH?$AAa?$AAl?$AAA?$AAl?$AAl?$AAo?$AAc?$AAa?$AAt?$AAe?$AAC?$AAo?$AAm?$AAm?$AAo?$AAn?$AAB?$AAu?$AAf?$AAf?$AAe?$AAr?$AA?3?$AA?5?$AAf?$AAa?$AAi?$AAl?$AAe?$AAd?$AA?5@ 10002008     ddk_dma:ddk_dma.obj
 0001:00001090       ??_C@_1II@KHPKJBHC@?$AAH?$AAa?$AAl?$AAA?$AAl?$AAl?$AAo?$AAc?$AAa?$AAt?$AAe?$AAC?$AAo?$AAm?$AAm?$AAo?$AAn?$AAB?$AAu?$AAf?$AAf?$AAe?$AAr?$AA?3?$AA?5?$AAm?$AAe?$AAm?$AAo?$AAr?$AAy?$AA?5@ 10002090     ddk_dma:ddk_dma.obj
 0001:00001118       ??_C@_1BA@LEPJIIOK@?$AAU?$AAn?$AAk?$AAn?$AAo?$AAw?$AAn?$AA?$AA@ 10002118     ddk_dma:ddk_dma.obj
 0001:00001128       ??_C@_1HK@FMKOKGJC@?$AAC?$AA?3?$AA?2?$AAy?$AAm?$AAz?$AAk?$AAi?$AA?2?$AAp?$AAu?$AAb?$AAl?$AAi?$AAc?$AA?2?$AAC?$AAO?$AAM?$AAM?$AAO?$AAN?$AA?2?$AAo?$AAa?$AAk?$AA?2?$AAd?$AAr?$AAi?$AAv?$AAe@ 10002128     ddk_dma:ddk_dma.obj
 0001:000011a8       ??_C@_1EM@IICCDICA@?$AAC?$AAe?$AAd?$AAd?$AAk?$AA?$CB?$AAB?$AAe?$AAg?$AAi?$AAn?$AAC?$AAa?$AAl?$AAi?$AAb?$AAr?$AAa?$AAt?$AAi?$AAo?$AAn?$AA?3?$AA?5?$AAD?$AAe?$AAl?$AAa?$AAy?$AA?5?$AAi?$AAs@ 100021a8     ddk_time:ddk_time.obj
 0001:000011f8       ??_C@_1LG@NACEBBBG@?$AAC?$AAe?$AAd?$AAd?$AAk?$AA?$CB?$AAB?$AAe?$AAg?$AAi?$AAn?$AAC?$AAa?$AAl?$AAi?$AAb?$AAr?$AAa?$AAt?$AAi?$AAo?$AAn?$AA?3?$AA?5?$AAC?$AAa?$AAl?$AAi?$AAb?$AAr?$AAa?$AAt@ 100021f8     ddk_time:ddk_time.obj
 0001:000012b0       ??_C@_1FA@GLLMJHHP@?$AAC?$AAe?$AAd?$AAd?$AAk?$AA?$CB?$AAB?$AAe?$AAg?$AAi?$AAn?$AAC?$AAa?$AAl?$AAi?$AAb?$AAr?$AAa?$AAt?$AAi?$AAo?$AAn?$AA?3?$AA?5?$AAE?$AAl?$AAa?$AAp?$AAs?$AAe?$AAd?$AA?5@ 100022b0     ddk_time:ddk_time.obj
 0001:00001300       ??_C@_1BE@PFMCPGJC@?$AAT?$AAh?$AAr?$AAe?$AAa?$AAd?$AAP?$AAr?$AAi?$AA?$AA@ 10002300     ddk_time:ddk_time.obj
 0001:00001318       ??_C@_1FE@EOKFGJML@?$AAC?$AAe?$AAd?$AAd?$AAk?$AA?$CB?$AAB?$AAe?$AAg?$AAi?$AAn?$AAC?$AAa?$AAl?$AAi?$AAb?$AAr?$AAa?$AAt?$AAi?$AAo?$AAn?$AA?3?$AA?5?$AAm?$AAi?$AAn?$AA?$CI?$AA?$CF?$AAd?$AA?$CJ?$AA?5@ 10002318     ddk_time:ddk_time.obj
 0001:00001370       ??_C@_1MK@BLLHFJNN@?$AAC?$AAe?$AAd?$AAd?$AAk?$AA?$CB?$AAB?$AAe?$AAg?$AAi?$AAn?$AAC?$AAa?$AAl?$AAi?$AAb?$AAr?$AAa?$AAt?$AAi?$AAo?$AAn?$AA?3?$AA?5?$AAF?$AAr?$AAe?$AAq?$AAu?$AAe?$AAn?$AAc@ 10002370     ddk_time:ddk_time.obj
 0001:00001440       ??_C@_1HO@MOGMJBMK@?$AAC?$AA?3?$AA?2?$AAy?$AAm?$AAz?$AAk?$AAi?$AA?2?$AAp?$AAu?$AAb?$AAl?$AAi?$AAc?$AA?2?$AAC?$AAO?$AAM?$AAM?$AAO?$AAN?$AA?2?$AAo?$AAa?$AAk?$AA?2?$AAd?$AAr?$AAi?$AAv?$AAe@ 10002440     ddk_time:ddk_time.obj
 0001:000014c0       ??_C@_1LE@JDNIKCBI@?$AAC?$AAe?$AAd?$AAd?$AAk?$AA?$CB?$AAB?$AAe?$AAg?$AAi?$AAn?$AAC?$AAa?$AAl?$AAi?$AAb?$AAr?$AAa?$AAt?$AAi?$AAo?$AAn?$AA?3?$AA?5?$AAP?$AAe?$AAr?$AAf?$AAo?$AAr?$AAm?$AAa@ 100024c0     ddk_time:ddk_time.obj
 0001:00001578       ??_C@_1IM@ILLHDHIF@?$AAC?$AAe?$AAd?$AAd?$AAk?$AA?$CB?$AAC?$AAa?$AAl?$AAi?$AAb?$AAr?$AAa?$AAt?$AAe?$AAS?$AAt?$AAa?$AAl?$AAl?$AAC?$AAo?$AAu?$AAn?$AAt?$AAe?$AAr?$AA?3?$AA?5?$AAS?$AAt?$AAa@ 10002578     ddk_time:ddk_time.obj
 0001:00001608       ??_C@_1HI@NGLAFFCK@?$AAC?$AAe?$AAd?$AAd?$AAk?$AA?$CB?$AAC?$AAa?$AAl?$AAi?$AAb?$AAr?$AAa?$AAt?$AAe?$AAS?$AAt?$AAa?$AAl?$AAl?$AAC?$AAo?$AAu?$AAn?$AAt?$AAe?$AAr?$AA?3?$AA?5?$AAC?$AAo?$AAu@ 10002608     ddk_time:ddk_time.obj
 0001:00001680       ??_C@_1GO@IDJCBAMN@?$AAC?$AAe?$AAd?$AAd?$AAk?$AA?$CB?$AAC?$AAa?$AAl?$AAi?$AAb?$AAr?$AAa?$AAt?$AAe?$AAS?$AAt?$AAa?$AAl?$AAl?$AAC?$AAo?$AAu?$AAn?$AAt?$AAe?$AAr?$AA?3?$AA?5?$AAN?$AAu?$AAm@ 10002680     ddk_time:ddk_time.obj
 0001:000016f0       ??_C@_1CG@KGDKIHGE@?$AAN?$AAu?$AAm?$AAC?$AAa?$AAl?$AAi?$AAb?$AAA?$AAc?$AAc?$AAe?$AAp?$AAt?$AAH?$AAi?$AAt?$AAs?$AA?$AA@ 100026f0     ddk_time:ddk_time.obj
 0001:00001718       ??_C@_1GK@PIDKDION@?$AAC?$AAe?$AAd?$AAd?$AAk?$AA?$CB?$AAC?$AAa?$AAl?$AAi?$AAb?$AAr?$AAa?$AAt?$AAe?$AAS?$AAt?$AAa?$AAl?$AAl?$AAC?$AAo?$AAu?$AAn?$AAt?$AAe?$AAr?$AA?3?$AA?5?$AAM?$AAa?$AAx@ 10002718     ddk_time:ddk_time.obj
 0001:00001784       ??_C@_1CC@LLDIACGB@?$AAM?$AAa?$AAx?$AAC?$AAa?$AAl?$AAi?$AAb?$AAA?$AAt?$AAt?$AAe?$AAm?$AAp?$AAt?$AAs?$AA?$AA@ 10002784     ddk_time:ddk_time.obj
 0001:000017a8       ??_C@_1GK@FLBPJBON@?$AAC?$AAe?$AAd?$AAd?$AAk?$AA?$CB?$AAC?$AAa?$AAl?$AAi?$AAb?$AAr?$AAa?$AAt?$AAe?$AAS?$AAt?$AAa?$AAl?$AAl?$AAC?$AAo?$AAu?$AAn?$AAt?$AAe?$AAr?$AA?3?$AA?5?$AAI?$AAn?$AAi@ 100027a8     ddk_time:ddk_time.obj
 0001:00001814       ??_C@_1CC@LCBAJDIB@?$AAI?$AAn?$AAi?$AAt?$AAS?$AAt?$AAa?$AAl?$AAl?$AAC?$AAo?$AAu?$AAn?$AAt?$AAe?$AAr?$AA?$AA@ 10002814     ddk_time:ddk_time.obj
 0001:00001838       ??_C@_1HI@GABKPNEA@?$AAC?$AAe?$AAd?$AAd?$AAk?$AA?$CB?$AAC?$AAa?$AAl?$AAi?$AAb?$AAr?$AAa?$AAt?$AAe?$AAS?$AAt?$AAa?$AAl?$AAl?$AAC?$AAo?$AAu?$AAn?$AAt?$AAe?$AAr?$AA?3?$AA?5?$AAC?$AAo?$AAu@ 10002838     ddk_time:ddk_time.obj
 0001:000018b0       ??_C@_1BK@EPHPAOMP@?$AAS?$AAt?$AAa?$AAl?$AAl?$AAC?$AAo?$AAu?$AAn?$AAt?$AAe?$AAr?$AA?$AA@ 100028b0     ddk_time:ddk_time.obj
 0001:000018cc       ??_C@_1CM@GACOAEOD@?$AAC?$AAa?$AAl?$AAi?$AAb?$AAr?$AAa?$AAt?$AAe?$AAS?$AAt?$AAa?$AAl?$AAl?$AAC?$AAo?$AAu?$AAn?$AAt?$AAe?$AAr?$AA?$AA@ 100028cc     ddk_time:ddk_time.obj
 0001:000018f8       ??_C@_1BK@OOAFBID@?$AAS?$AAy?$AAs?$AAt?$AAe?$AAm?$AA?2?$AAC?$AAe?$AAd?$AAd?$AAk?$AA?$AA@ 100028f8     ddk_time:ddk_time.obj
 0001:00001918       ??_C@_1IE@HEEDGCIH@?$AAC?$AAe?$AAd?$AAd?$AAk?$AA?$CB?$AAC?$AAa?$AAl?$AAi?$AAb?$AAr?$AAa?$AAt?$AAe?$AAS?$AAt?$AAa?$AAl?$AAl?$AAC?$AAo?$AAu?$AAn?$AAt?$AAe?$AAr?$AA?3?$AA?5?$AAG?$AAe?$AAt@ 10002918     ddk_time:ddk_time.obj
 0001:0000199c       ??_C@_1BO@FJAFIJCI@?$AAR?$AAe?$AAg?$AAS?$AAe?$AAt?$AAV?$AAa?$AAl?$AAu?$AAe?$AAE?$AAx?$AAW?$AA?$AA@ 1000299c     ddk_time:ddk_time.obj
 0001:000019bc       ??_C@_1CC@KOJKGDIE@?$AAR?$AAe?$AAg?$AAQ?$AAu?$AAe?$AAr?$AAy?$AAV?$AAa?$AAl?$AAu?$AAe?$AAE?$AAx?$AAW?$AA?$AA@ 100029bc     ddk_time:ddk_time.obj
 0001:000019e0       ??_C@_1BI@FBGIJHPE@?$AAR?$AAe?$AAg?$AAC?$AAl?$AAo?$AAs?$AAe?$AAK?$AAe?$AAy?$AA?$AA@ 100029e0     ddk_time:ddk_time.obj
 0001:000019f8       ??_C@_1CA@DDPBCKNC@?$AAR?$AAe?$AAg?$AAC?$AAr?$AAe?$AAa?$AAt?$AAe?$AAK?$AAe?$AAy?$AAE?$AAx?$AAW?$AA?$AA@ 100029f8     ddk_time:ddk_time.obj
 0001:00001a18       ??_C@_1BI@CJKPFBEK@?$AAc?$AAo?$AAr?$AAe?$AAd?$AAl?$AAl?$AA?4?$AAd?$AAl?$AAl?$AA?$AA@ 10002a18     ddk_time:ddk_time.obj
 0001:00001a30       ??_C@_1EK@EACPGFCN@?$AAC?$AAe?$AAd?$AAd?$AAk?$AA?$CB?$AAC?$AAa?$AAl?$AAi?$AAb?$AAr?$AAa?$AAt?$AAe?$AAS?$AAt?$AAa?$AAl?$AAl?$AAC?$AAo?$AAu?$AAn?$AAt?$AAe?$AAr?$AA?3?$AA?5?$AAE?$AAn?$AAt@ 10002a30     ddk_time:ddk_time.obj
 0001:00001b10       ??_C@_1DO@KCLIIBNE@?$AAV?$AAi?$AAr?$AAt?$AAu?$AAa?$AAl?$AAS?$AAe?$AAt?$AAA?$AAt?$AAt?$AAr?$AAi?$AAb?$AAu?$AAt?$AAe?$AAs?$AA?5?$AAf?$AAa?$AAi?$AAl?$AAe?$AAd?$AA?$CB?$AA?$AN?$AA?6?$AA?$AA@ 10002b10     ddk_sdma:ddk_sdma.obj
 0001:00001b50       ??_C@_1KK@PBHBAOKF@?$AAC?$AA?3?$AA?2?$AAW?$AAI?$AAN?$AAC?$AAE?$AAR?$AAO?$AAO?$AAT?$AAS?$AA?2?$AAT?$AAo?$AAp?$AAa?$AAz?$AA?2?$AAW?$AAI?$AAN?$AAC?$AAE?$AA6?$AA0?$AA0?$AA?2?$AAP?$AAL?$AAA@ 10002b50     ddk_sdma:ddk_sdma.obj
 0001:00001c20       ClockInit                  10002c20 f   ddk_mx25_topaz_v1:soc_ddk_clk.obj
 0001:00001c38       ClockAlloc                 10002c38 f   ddk_mx25_topaz_v1:soc_ddk_clk.obj
 0001:00001d30       ClockDealloc               10002d30 f   ddk_mx25_topaz_v1:soc_ddk_clk.obj
 0001:00001d94       DDKClockSetGatingMode      10002d94 f   ddk_mx25_topaz_v1:soc_ddk_clk.obj
 0001:00001ec4       DDKClockGetGatingMode      10002ec4 f   ddk_mx25_topaz_v1:soc_ddk_clk.obj
 0001:00001f3c       DDKClockGetFreq            10002f3c f   ddk_mx25_topaz_v1:soc_ddk_clk.obj
 0001:00001f74       DDKClockConfigBaud         10002f74 f   ddk_mx25_topaz_v1:soc_ddk_clk.obj
 0001:000021a0       DDKClockSetCKO             100031a0 f   ddk_mx25_topaz_v1:soc_ddk_clk.obj
 0001:0000224c       DDKClockSetpointRequest    1000324c f   ddk_mx25_topaz_v1:soc_ddk_clk.obj
 0001:00002284       DDKClockSetpointRelease    10003284 f   ddk_mx25_topaz_v1:soc_ddk_clk.obj
 0001:000022b8       DDKClockGetSharedConfig    100032b8 f   ddk_mx25_topaz_v1:soc_ddk_clk.obj
 0001:000022d8       DDKClockLock               100032d8 f   ddk_mx25_topaz_v1:soc_ddk_clk.obj
 0001:000022f0       DDKClockUnlock             100032f0 f   ddk_mx25_topaz_v1:soc_ddk_clk.obj
 0001:00002308       DDKGpioSetConfig           10003308 f   ddk_mx25_topaz_v1:ddk_gpio.obj
 0001:0000277c       DDKGpioGetConfig           1000377c f   ddk_mx25_topaz_v1:ddk_gpio.obj
 0001:000029cc       DDKGpioWriteData           100039cc f   ddk_mx25_topaz_v1:ddk_gpio.obj
 0001:00002ae4       DDKGpioWriteDataPin        10003ae4 f   ddk_mx25_topaz_v1:ddk_gpio.obj
 0001:00002b84       DDKGpioReadData            10003b84 f   ddk_mx25_topaz_v1:ddk_gpio.obj
 0001:00002c54       DDKGpioReadDataPin         10003c54 f   ddk_mx25_topaz_v1:ddk_gpio.obj
 0001:00002d20       DDKGpioReadIntr            10003d20 f   ddk_mx25_topaz_v1:ddk_gpio.obj
 0001:00002df0       DDKGpioReadIntrPin         10003df0 f   ddk_mx25_topaz_v1:ddk_gpio.obj
 0001:00002ebc       DDKGpioClearIntr           10003ebc f   ddk_mx25_topaz_v1:ddk_gpio.obj
 0001:00002f80       DDKGpioClearIntrPin        10003f80 f   ddk_mx25_topaz_v1:ddk_gpio.obj
 0001:00003074       GpioDealloc                10004074 f   ddk_mx25_topaz_v1:ddk_gpio.obj
 0001:00003128       GpioAlloc                  10004128 f   ddk_mx25_topaz_v1:ddk_gpio.obj
 0001:00003280       DDKIomuxSetPinMux          10004280 f   ddk_mx25_topaz_v1:soc_ddk_iomux.obj
 0001:000032d8       DDKIomuxGetPinMux          100042d8 f   ddk_mx25_topaz_v1:soc_ddk_iomux.obj
 0001:00003348       DDKIomuxSetPadConfig       10004348 f   ddk_mx25_topaz_v1:soc_ddk_iomux.obj
 0001:000033c0       DDKIomuxGetPadConfig       100043c0 f   ddk_mx25_topaz_v1:soc_ddk_iomux.obj
 0001:00003470       DDKIomuxSetPadConfigPort   10004470 f   ddk_mx25_topaz_v1:soc_ddk_iomux.obj
 0001:000034c0       DDKIomuxGetPadConfigPort   100044c0 f   ddk_mx25_topaz_v1:soc_ddk_iomux.obj
 0001:00003514       DDKIomuxSelectInput        10004514 f   ddk_mx25_topaz_v1:soc_ddk_iomux.obj
 0001:00003564       IomuxAlloc                 10004564 f   ddk_mx25_topaz_v1:soc_ddk_iomux.obj
 0001:00003650       IomuxDealloc               10004650 f   ddk_mx25_topaz_v1:soc_ddk_iomux.obj
 0001:000036a4       DDKSdmaOpenChan            100046a4 f   ddk_mx25_topaz_v1:ddk_sdmav2.obj
 0001:00003a84       DDKSdmaUpdateSharedChan    10004a84 f   ddk_mx25_topaz_v1:ddk_sdmav2.obj
 0001:00003b2c       DDKSdmaCloseChan           10004b2c f   ddk_mx25_topaz_v1:ddk_sdmav2.obj
 0001:00003e6c       DDKSdmaAllocChain          10004e6c f   ddk_mx25_topaz_v1:ddk_sdmav2.obj
 0001:00003fd4       DDKSdmaFreeChain           10004fd4 f   ddk_mx25_topaz_v1:ddk_sdmav2.obj
 0001:000041a0       DDKSdmaSetBufDesc          100051a0 f   ddk_mx25_topaz_v1:ddk_sdmav2.obj
 0001:000043c4       DDKSdmaGetBufDescStatus    100053c4 f   ddk_mx25_topaz_v1:ddk_sdmav2.obj
 0001:0000455c       DDKSdmaGetChainStatus      1000555c f   ddk_mx25_topaz_v1:ddk_sdmav2.obj
 0001:00004760       DDKSdmaClearBufDescStatus  10005760 f   ddk_mx25_topaz_v1:ddk_sdmav2.obj
 0001:00004a64       DDKSdmaClearChainStatus    10005a64 f   ddk_mx25_topaz_v1:ddk_sdmav2.obj
 0001:00004db0       DDKSdmaInitChain           10005db0 f   ddk_mx25_topaz_v1:ddk_sdmav2.obj
 0001:00004f70       DDKSdmaStartChan           10005f70 f   ddk_mx25_topaz_v1:ddk_sdmav2.obj
 0001:0000509c       DDKSdmaStopChan            1000609c f   ddk_mx25_topaz_v1:ddk_sdmav2.obj
 0001:00005150       SdmaInit                   10006150 f   ddk_mx25_topaz_v1:ddk_sdmav2.obj
 0001:00005344       SdmaDeinit                 10006344 f   ddk_mx25_topaz_v1:ddk_sdmav2.obj
 0001:000053a4       SdmaAlloc                  100063a4 f   ddk_mx25_topaz_v1:ddk_sdmav2.obj
 0001:000055f8       SdmaDealloc                100065f8 f   ddk_mx25_topaz_v1:ddk_sdmav2.obj
 0001:00005e4c       DllEntry                   10006e4c f   ddk_mx25_topaz_v1:cspddk.obj
 0001:00005f9c       Init                       10006f9c f   ddk_mx25_topaz_v1:cspddk.obj
 0001:00006008       Deinit                     10007008 f   ddk_mx25_topaz_v1:cspddk.obj
 0001:00006038       SdmaLoadRamScripts         10007038 f   ddk_mx25_topaz_v1:soc_ddk_sdma.obj
 0001:0000607c       SdmaSetChanDesc            1000707c f   ddk_mx25_topaz_v1:soc_ddk_sdma.obj
 0001:00006ebc       SdmaUpdateChanDesc         10007ebc f   ddk_mx25_topaz_v1:soc_ddk_sdma.obj
 0001:00006ee4       SdmaSetChanContext         10007ee4 f   ddk_mx25_topaz_v1:soc_ddk_sdma.obj
 0001:00007078       BSPClockDealloc            10008078 f   ddk_clk:ddk_clk.obj
 0001:00007150       BSPClockAlloc              10008150 f   ddk_clk:ddk_clk.obj
 0001:000073c8       BSPClockGetFreq            100083c8 f   ddk_clk:ddk_clk.obj
 0001:0000741c       BSPClockUpdateFreq         1000841c f   ddk_clk:ddk_clk.obj
 0001:0000756c       BSPClockSetGatingModePrepare 1000856c f   ddk_clk:ddk_clk.obj
 0001:00007594       BSPClockSetGatingModeComplete 10008594 f   ddk_clk:ddk_clk.obj
 0001:000076ac       BSPClockSetpointRequest    100086ac f   ddk_clk:ddk_clk.obj
 0001:000077d4       BSPClockSetpointRelease    100087d4 f   ddk_clk:ddk_clk.obj
 0001:00007874       ResetEvent                 10008874 f i ddk_clk:ddk_clk.obj
 0001:000078ac       SetEvent                   100088ac f i ddk_clk:ddk_clk.obj
 0001:000078e4       HalAllocateCommonBuffer    100088e4 f   ddk_dma:ddk_dma.obj
 0001:00007a44       HalFreeCommonBuffer        10008a44 f   ddk_dma:ddk_dma.obj
 0001:00007a78       GetDMAAdapterHandle        10008a78 f   ddk_dma:ddk_dma.obj
 0001:00007be4       DMAGetAdapter              10008be4 f   ddk_dma:ddk_dma.obj
 0001:00007c7c       DMAAllocateChannel         10008c7c f   ddk_dma:ddk_dma.obj
 0001:00007d78       DMAFreeChannel             10008d78 f   ddk_dma:ddk_dma.obj
 0001:00007e18       DMAIssueTransfer           10008e18 f   ddk_dma:ddk_dma.obj
 0001:00007f60       DMAIssueMultiBufferTransfer 10008f60 f   ddk_dma:ddk_dma.obj
 0001:0000809c       DMACancelTransfer          1000909c f   ddk_dma:ddk_dma.obj
 0001:00008180       DMAStartTransfer           10009180 f   ddk_dma:ddk_dma.obj
 0001:00008264       DMACloseTransfer           10009264 f   ddk_dma:ddk_dma.obj
 0001:0000834c       DMAGetStatus               1000934c f   ddk_dma:ddk_dma.obj
 0001:00008438       DMAGetContexts             10009438 f   ddk_dma:ddk_dma.obj
 0001:00008524       DMAIssueRawTransfer        10009524 f   ddk_dma:ddk_dma.obj
 0001:00008648       DMARawTransferControl      10009648 f   ddk_dma:ddk_dma.obj
 0001:00008708       OALDMAAllocBuffer          10009708 f   ddk_dma:ddk_dma.obj
 0001:00008848       OALDMAFreeBuffer           10009848 f   ddk_dma:ddk_dma.obj
 0001:00008944       MmMapIoSpace               10009944 f   ddk_map:ddk_map.obj
 0001:00008ac4       MmUnmapIoSpace             10009ac4 f   ddk_map:ddk_map.obj
 0001:00008b00       TransBusAddrToVirtual      10009b00 f   ddk_map:ddk_map.obj
 0001:00008bc8       TransBusAddrToStatic       10009bc8 f   ddk_map:ddk_map.obj
 0001:00008d24       StallOneMicrosecond        10009d24 f   ddk_time:ddk_time.obj
 0001:00008d74       BeginCalibration           10009d74 f   ddk_time:ddk_time.obj
 0001:00009180       CalibrateStallCounter      1000a180 f   ddk_time:ddk_time.obj
 0001:000095bc       StallExecution             1000a5bc f   ddk_time:ddk_time.obj
 0001:000096f0       GetCurrentThread           1000a6f0 f i ddk_time:ddk_time.obj
 0001:00009708       BSPSdmaAllocShared         1000a708 f   ddk_sdma:ddk_sdma.obj
 0001:00009874       BSPSdmaAllocChain          1000a874 f   ddk_sdma:ddk_sdma.obj
 0001:00009a98       BSPSdmaFreeChain           1000aa98 f   ddk_sdma:ddk_sdma.obj
 0001:00009b60       BSPSdmaBufIntMem           1000ab60 f   ddk_sdma:ddk_sdma.obj
 0001:00009be4       BSPSdmaGetM3BaseAddr       1000abe4 f   ddk_sdma:ddk_sdma.obj
 0001:00009bfc       InitializeCriticalSection  1000abfc f   coredll:COREDLL.dll
 0001:00009c0c       NKDbgPrintfW               1000ac0c f   coredll:COREDLL.dll
 0001:00009c1c       DeleteCriticalSection      1000ac1c f   coredll:COREDLL.dll
 0001:00009c2c       LeaveCriticalSection       1000ac2c f   coredll:COREDLL.dll
 0001:00009c3c       EnterCriticalSection       1000ac3c f   coredll:COREDLL.dll
 0001:00009c4c       InterlockedCompareExchange 1000ac4c f   coredll:COREDLL.dll
 0001:00009c5c       ReleaseMutex               1000ac5c f   coredll:COREDLL.dll
 0001:00009c6c       WaitForSingleObject        1000ac6c f   coredll:COREDLL.dll
 0001:00009c7c       CreateMutexW               1000ac7c f   coredll:COREDLL.dll
 0001:00009c8c       CloseHandle                1000ac8c f   coredll:COREDLL.dll
 0001:00009c9c       Sleep                      1000ac9c f   coredll:COREDLL.dll
 0001:00009cac       DisableThreadLibraryCalls  1000acac f   coredll:COREDLL.dll
 0001:00009cbc       CreateEventW               1000acbc f   coredll:COREDLL.dll
 0001:00009ccc       InterlockedIncrement       1000accc f   coredll:COREDLL.dll
 0001:00009cdc       EventModify                1000acdc f   coredll:COREDLL.dll
 0001:00009cec       InterlockedDecrement       1000acec f   coredll:COREDLL.dll
 0001:00009cfc       FreePhysMem                1000acfc f   coredll:COREDLL.dll
 0001:00009d0c       GetLastError               1000ad0c f   coredll:COREDLL.dll
 0001:00009d1c       AllocPhysMem               1000ad1c f   coredll:COREDLL.dll
 0001:00009d2c       InterlockedExchange        1000ad2c f   coredll:COREDLL.dll
 0001:00009d3c       CreateFileW                1000ad3c f   coredll:COREDLL.dll
 0001:00009d4c       RegCloseKey                1000ad4c f   coredll:COREDLL.dll
 0001:00009d5c       RegQueryValueExW           1000ad5c f   coredll:COREDLL.dll
 0001:00009d6c       RegOpenKeyExW              1000ad6c f   coredll:COREDLL.dll
 0001:00009d7c       DeviceIoControl            1000ad7c f   coredll:COREDLL.dll
 0001:00009d8c       SetLastError               1000ad8c f   coredll:COREDLL.dll
 0001:00009d9c       VirtualFree                1000ad9c f   coredll:COREDLL.dll
 0001:00009dac       VirtualCopy                1000adac f   coredll:COREDLL.dll
 0001:00009dbc       VirtualAlloc               1000adbc f   coredll:COREDLL.dll
 0001:00009dcc       CreateStaticMapping        1000adcc f   coredll:COREDLL.dll
 0001:00009ddc       CeSetThreadPriority        1000addc f   coredll:COREDLL.dll
 0001:00009dec       QueryPerformanceCounter    1000adec f   coredll:COREDLL.dll
 0001:00009dfc       QueryPerformanceFrequency  1000adfc f   coredll:COREDLL.dll
 0001:00009e0c       CeGetThreadPriority        1000ae0c f   coredll:COREDLL.dll
 0001:00009e1c       FreeLibrary                1000ae1c f   coredll:COREDLL.dll
 0001:00009e2c       GetProcAddressW            1000ae2c f   coredll:COREDLL.dll
 0001:00009e3c       LoadLibraryW               1000ae3c f   coredll:COREDLL.dll
 0001:00009e4c       CacheRangeFlush            1000ae4c f   coredll:COREDLL.dll
 0001:00009e5c       VirtualSetAttributes       1000ae5c f   coredll:COREDLL.dll
 0001:00009e6c       _DllEntryCRTStartup        1000ae6c f   corelib0:pegdentry.obj
 0001:00009edc       __security_init_cookie     1000aedc f   corelib0:seccinit.obj
 0001:00009fa4       __GSHandlerCheck           1000afa4 f   corelib0:gshandler.obj
 0001:00009fec       __GSHandlerCheckCommon     1000afec f   corelib0:gshandler.obj
 0001:0000a094       __security_check_cookie    1000b094 f   corelib0:armsecgs.obj
 0001:0000a0a8       __gsfailure                1000b0a8 f   corelib0:armsecgs.obj
 0001:0000a0ec       exit                       1000b0ec f   corelib0:cexit.obj
 0001:0000a26c       _exit                      1000b26c f   corelib0:cexit.obj
 0001:0000a290       _cexit                     1000b290 f   corelib0:cexit.obj
 0001:0000a2ac       _c_exit                    1000b2ac f   corelib0:cexit.obj
 0001:0000a2c8       GetCurrentProcess          1000b2c8 f i corelib0:cexit.obj
 0001:0000a2e0       _initterm                  1000b2e0 f   corelib0:crt0dat.obj
 0001:0000a334       _cinit                     1000b334 f   corelib0:crt0dat.obj
 0001:0000a370       _onexit                    1000b370 f   corelib0:onexit.obj
 0001:0000a674       atexit                     1000b674 f   corelib0:onexit.obj
 0001:0000a6c8       memset                     1000b6c8 f   corelib1:COREDLL.dll
 0001:0000a6d8       __rt_sdiv                  1000b6d8 f   corelib1:COREDLL.dll
 0001:0000a6e8       memcpy                     1000b6e8 f   corelib1:COREDLL.dll
 0001:0000a6f8       __rt_udiv                  1000b6f8 f   corelib1:COREDLL.dll
 0001:0000a708       __rt_sdiv64by64            1000b708 f   corelib1:COREDLL.dll
 0001:0000a718       __security_gen_cookie2     1000b718 f   corelib1:COREDLL.dll
 0001:0000a728       __report_gsfailure         1000b728 f   corelib1:COREDLL.dll
 0001:0000a738       free                       1000b738 f   corelib1:COREDLL.dll
 0001:0000a748       __C_specific_handler       1000b748 f   corelib1:COREDLL.dll
 0001:0000a758       malloc                     1000b758 f   corelib1:COREDLL.dll
 0001:0000a768       realloc                    1000b768 f   corelib1:COREDLL.dll
 0001:0000a778       _msize                     1000b778 f   corelib1:COREDLL.dll
 0001:0000a788       HalGetBusDataByOffset      1000b788 f   ddk_bus:ddk_bus.obj
 0001:0000a7b0       HalSetBusDataByOffset      1000b7b0 f   ddk_bus:ddk_bus.obj
 0001:0000a7d8       HalTranslateBusAddress     1000b7d8 f   ddk_bus:ddk_bus.obj
 0001:0000a81c       HalTranslateSystemAddress  1000b81c f   ddk_bus:ddk_bus.obj
 0001:0000a874       TerminateProcess           1000b874 f   coredll:COREDLL.dll
 0001:0000a89c       __IMPORT_DESCRIPTOR_COREDLL 1000b89c     coredll:COREDLL.dll
 0001:0000a8b0       __NULL_IMPORT_DESCRIPTOR   1000b8b0     coredll:COREDLL.dll
 0002:00000000       __imp_InitializeCriticalSection 1000c000     coredll:COREDLL.dll
 0002:00000004       __imp_NKDbgPrintfW         1000c004     coredll:COREDLL.dll
 0002:00000008       __imp_DeleteCriticalSection 1000c008     coredll:COREDLL.dll
 0002:0000000c       __imp_LeaveCriticalSection 1000c00c     coredll:COREDLL.dll
 0002:00000010       __imp_EnterCriticalSection 1000c010     coredll:COREDLL.dll
 0002:00000014       __imp_InterlockedCompareExchange 1000c014     coredll:COREDLL.dll
 0002:00000018       __imp_ReleaseMutex         1000c018     coredll:COREDLL.dll
 0002:0000001c       __imp_WaitForSingleObject  1000c01c     coredll:COREDLL.dll
 0002:00000020       __imp_CreateMutexW         1000c020     coredll:COREDLL.dll
 0002:00000024       __imp_CloseHandle          1000c024     coredll:COREDLL.dll
 0002:00000028       __imp_Sleep                1000c028     coredll:COREDLL.dll
 0002:0000002c       __imp_DisableThreadLibraryCalls 1000c02c     coredll:COREDLL.dll
 0002:00000030       __imp_CreateEventW         1000c030     coredll:COREDLL.dll
 0002:00000034       __imp_InterlockedIncrement 1000c034     coredll:COREDLL.dll
 0002:00000038       __imp_EventModify          1000c038     coredll:COREDLL.dll
 0002:0000003c       __imp_InterlockedDecrement 1000c03c     coredll:COREDLL.dll
 0002:00000040       __imp_FreePhysMem          1000c040     coredll:COREDLL.dll
 0002:00000044       __imp_GetLastError         1000c044     coredll:COREDLL.dll
 0002:00000048       __imp_AllocPhysMem         1000c048     coredll:COREDLL.dll
 0002:0000004c       __imp_InterlockedExchange  1000c04c     coredll:COREDLL.dll
 0002:00000050       __imp_CreateFileW          1000c050     coredll:COREDLL.dll
 0002:00000054       __imp_RegCloseKey          1000c054     coredll:COREDLL.dll
 0002:00000058       __imp_RegQueryValueExW     1000c058     coredll:COREDLL.dll
 0002:0000005c       __imp_RegOpenKeyExW        1000c05c     coredll:COREDLL.dll
 0002:00000060       __imp_DeviceIoControl      1000c060     coredll:COREDLL.dll
 0002:00000064       __imp_SetLastError         1000c064     coredll:COREDLL.dll
 0002:00000068       __imp_VirtualFree          1000c068     coredll:COREDLL.dll
 0002:0000006c       __imp_VirtualCopy          1000c06c     coredll:COREDLL.dll
 0002:00000070       __imp_VirtualAlloc         1000c070     coredll:COREDLL.dll
 0002:00000074       __imp_CreateStaticMapping  1000c074     coredll:COREDLL.dll
 0002:00000078       __imp_CeSetThreadPriority  1000c078     coredll:COREDLL.dll
 0002:0000007c       __imp_QueryPerformanceCounter 1000c07c     coredll:COREDLL.dll
 0002:00000080       __imp_QueryPerformanceFrequency 1000c080     coredll:COREDLL.dll
 0002:00000084       __imp_CeGetThreadPriority  1000c084     coredll:COREDLL.dll
 0002:00000088       __imp_FreeLibrary          1000c088     coredll:COREDLL.dll
 0002:0000008c       __imp_GetProcAddressW      1000c08c     coredll:COREDLL.dll
 0002:00000090       __imp_LoadLibraryW         1000c090     coredll:COREDLL.dll
 0002:00000094       __imp_CacheRangeFlush      1000c094     coredll:COREDLL.dll
 0002:00000098       __imp_VirtualSetAttributes 1000c098     coredll:COREDLL.dll
 0002:0000009c       __imp_memset               1000c09c     corelib1:COREDLL.dll
 0002:000000a0       __imp___rt_sdiv            1000c0a0     corelib1:COREDLL.dll
 0002:000000a4       __imp_memcpy               1000c0a4     corelib1:COREDLL.dll
 0002:000000a8       __imp___rt_udiv            1000c0a8     corelib1:COREDLL.dll
 0002:000000ac       __imp___rt_sdiv64by64      1000c0ac     corelib1:COREDLL.dll
 0002:000000b0       __imp___security_gen_cookie2 1000c0b0     corelib1:COREDLL.dll
 0002:000000b4       __imp___report_gsfailure   1000c0b4     corelib1:COREDLL.dll
 0002:000000b8       __imp_free                 1000c0b8     corelib1:COREDLL.dll
 0002:000000bc       __imp___C_specific_handler 1000c0bc     corelib1:COREDLL.dll
 0002:000000c0       __imp_malloc               1000c0c0     corelib1:COREDLL.dll
 0002:000000c4       __imp_realloc              1000c0c4     corelib1:COREDLL.dll
 0002:000000c8       __imp__msize               1000c0c8     corelib1:COREDLL.dll
 0002:000000cc       __imp_TerminateProcess     1000c0cc     coredll:COREDLL.dll
 0002:000000d0       \177COREDLL_NULL_THUNK_DATA 1000c0d0     coredll:COREDLL.dll
 0002:000000d8       g_DmaAdapter               1000c0d8     ddk_mx25_topaz_v1:ddk_sdmav2.obj
 0002:000000e8       g_SupportBothEdgeIntr      1000c0e8     ddk_mx25_topaz_v1:soc_ddk_gpio.obj
 0002:000000ec       g_MaxPort                  1000c0ec     ddk_mx25_topaz_v1:soc_ddk_gpio.obj
 0002:000000f0       g_PhyBaseAddress           1000c0f0     ddk_mx25_topaz_v1:soc_ddk_gpio.obj
 0002:00000110       g_hDma                     1000c110     ddk_dma:ddk_dma.obj
 0002:00000114       __security_cookie          1000c114     corelib0:seccinit.obj
 0002:00000118       __security_cookie_complement 1000c118     corelib0:seccinit.obj
 0002:00000120       g_pCRM                     1000c120     ddk_mx25_topaz_v1:soc_ddk_clk.obj
 0002:00000124       g_pDdkClkConfig            1000c124     ddk_mx25_topaz_v1:soc_ddk_clk.obj
 0002:00000134       g_pHostSharedUA            1000c134     ddk_mx25_topaz_v1:ddk_sdmav2.obj
 0002:00000138       g_pHostSharedPA            1000c138     ddk_mx25_topaz_v1:ddk_sdmav2.obj
 0002:0000013c       g_HostSharedSize           1000c13c     ddk_mx25_topaz_v1:ddk_sdmav2.obj
 0002:00000160       _exitflag                  1000c160     corelib0:cexit.obj
 0002:00000170       g_pGPIO                    1000c170     <common>
 0002:00000180       g_csDdkClk                 1000c180     <common>
 0002:00000194       g_NumCalibAcceptHits       1000c194     <common>
 0002:00000198       g_fStallCounterSet         1000c198     <common>
 0002:0000019c       g_StallCounter             1000c19c     <common>
 0002:000001a0       g_InitStallCounter         1000c1a0     <common>
 0002:000001a4       g_MaxCalibAttempts         1000c1a4     <common>
 0002:000001a8       g_StallDummy               1000c1a8     <common>
 0002:000001ac       __onexitend                1000c1ac     <common>
 0002:000001b0       __onexitbegin              1000c1b0     <common>
 0002:000001b4       g_pcsExit                  1000c1b4     <common>

 entry point at        0001:00009e6c

 Static symbols

 0001:000056e8       SdmaWritePM                100066e8 f   ddk_mx25_topaz_v1:ddk_sdmav2.obj
 0001:00005878       SdmaWriteChanContext       10006878 f   ddk_mx25_topaz_v1:ddk_sdmav2.obj
 0001:000059e8       SdmaSetChanOverride        100069e8 f   ddk_mx25_topaz_v1:ddk_sdmav2.obj
 0001:00005b64       SdmaSetChanPriority        10006b64 f   ddk_mx25_topaz_v1:ddk_sdmav2.obj
 0001:00005ba4       SdmaGetChanStatus          10006ba4 f   ddk_mx25_topaz_v1:ddk_sdmav2.obj
 0001:00005c0c       SdmaFindUnusedChan         10006c0c f   ddk_mx25_topaz_v1:ddk_sdmav2.obj
 0001:00005d10       SdmaLockCtrlChan           10006d10 f   ddk_mx25_topaz_v1:ddk_sdmav2.obj
 0001:00005d48       SdmaUnlockCtrlChan         10006d48 f   ddk_mx25_topaz_v1:ddk_sdmav2.obj
 0001:00005d7c       SdmaValidChan              10006d7c f   ddk_mx25_topaz_v1:ddk_sdmav2.obj
 0001:0000a110       doexit                     1000b110 f   corelib0:cexit.obj
 0001:0000a3cc       lockexit                   1000b3cc f   corelib0:onexit.obj
 0001:0000a468       unlockexit                 1000b468 f   corelib0:onexit.obj
 0001:0000a494       _onexit_nolock             1000b494 f   corelib0:onexit.obj
